:1000000012C02DC02CC02BC02AC029C028C027C0B8
:1000100026C025C024C023C022C021C020C01FC0CC
:100020001EC06A62000011241FBECFE5D1E0DEBF12
:10003000CDBF10E0A0E6B0E0ECECF2E003C0C89564
:1000400031960D92A036B107D1F710E0A0E6B0E0EE
:1000500001C01D92A036B107E1F7F9D036C1D0CF6B
:10006000982F9095D8988AE88A95F1F7292F332709
:1000700027FD309520FF02C0D89801C0D89A8AE8A1
:100080008A95F1F721FF02C0D89801C0D89A8AE872
:100090008A95F1F722FF02C0D89801C0D89A8AE861
:1000A0008A95F1F723FF02C0D89801C0D89A8AE850
:1000B0008A95F1F724FF02C0D89801C0D89A8AE83F
:1000C0008A95F1F725FF02C0D89801C0D89A8AE82E
:1000D0008A95F1F726FF02C0D89801C0D89A8AE81D
:1000E0008A95F1F797FF02C0D89801C0D89A8AE89C
:1000F000982F9A95F1F7D89A8A95F1F70895CF93AA
:10010000DF93D92FC82FF92FE82F2196C895802D7E
:10011000882341F0A5DFFD2FEC2F2196C895802D77
:100120008823C1F7DF91CF91089582E0982F9A95A7
:10013000F1F7DC988A95F1F7DC9A0895EF92FF9237
:100140000F931F93CF93DF93082F192FE62EF72ECF
:10015000D69ADE9AEADF0038110514F000581040F4
:10016000C6E0D0E0912F802F0C2E02C09595879588
:100170000A94E2F780FF02C0DE9A01C0DE98D5DF64
:100180002197D7FFEFCFC7E0D0E09F2D8E2D0C2E0B
:1001900002C0959587950A94E2F780FF02C0DE9A27
:1001A00001C0DE98C2DF2197D7FFEFCFDF91CF915B
:1001B0001F910F91FF90EF900895EF92FF920F9390
:1001C0001F93CF93DF93082F192FEE24FF24D69A85
:1001D000DE98ABDF0038110514F000581040C6E07F
:1001E000D0E0912F802F0C2E02C0959587950A9410
:1001F000E2F780FF02C0DE9A01C0DE9896DF219709
:10020000D7FFEFCF8CE291E00197F1F7D698DE9817
:10021000C7E0D0E08ADF82E08A95F1F7CE9B0AC082
:1002200081E090E00C2E02C0880F991F0A94E2F73B
:10023000E82AF92A2197D7FFEDCFDC989F2D8E2D44
:10024000DF91CF911F910F91FF90EF900895CFE52F
:10025000D1E0DEBFCDBF80E886BD16BC28EE33E01E
:1002600088EC90E00197F1F721503040C9F7D09A1F
:10027000D898D49ADC9A60E070E088E090E05EDF85
:1002800000E010E0C1E1D0E080EA9FE00197F1F7E3
:1002900088E090E092DF86FF02C08F7301C081E8A2
:1002A000DFDE2197D7FFF0CF0F5F1F4F023111051F
:1002B0004CF380E8D5DE28EE33E088EC90E001973F
:0C02C000F1F721503040C9F7D6CFFFCF36
:00000001FF
